:020000000134C9
:20003400758171758901D2AFD28C1204C212001B80FB0581740A75F000C0E0C0F074027543
:20005400F000C0E0C0F01207BF15811581158115815480C5F05400C5F078FE122895F6450A
:20007400F07003020098E61228C77BFF1228BE1229C845F0700302009574FF75F0FF0200FB
:200094009D020048740175F000158122120046740A75F000C0E0C0F0740075F000C0E0C00F
:2000B400F0740175F000C0E0C0F01207E87FFA1228A1221200467BFF7CFF1229C845F070A6
:2000D400030200E074FF75F0FF020149740A75F000C0E0C0F0740075F000C0E0C0F07438FC
:2000F40075F000C0E0C0F01207E87FFA1228A1120046740A75F000C0E0C0F0740075F0007E
:20011400C0E0C0F0740C75F000C0E0C0F01207E87FFA1228A11200A0740075F000C0E0C006
:20013400F0740075F000C0E0C0F012014A15811581158115812212004678FB122895E61229
:2001540028C790020C0228D0740A75F000C0E0C0F0740075F000C0E0C0F078F5122895E686
:2001740024801228C7C0E0C0F01207E87FFA1228A1020220740A75F000C0E0C0F0740075E1
:20019400F000C0E0C0F078F5122895E624C01228C7C0E0C0F01207E87FFA1228A10202203B
:2001B400740A75F000C0E0C0F0740075F000C0E0C0F078F5122895E624941228C7C0E0C094
:2001D400F01207E87FFA1228A1020220740A75F000C0E0C0F0740075F000C0E0C0F078F5D9
:2001F400122895E624D41228C7C0E0C0F01207E87FFA1228A1020220E0010300B4010200D9
:20021400880101005C01000000002002220581740078FE122895F678FE122895E6181818F7
:2002340018860108860275F0001228B789828A83E4931228C77B001228BE1229D145F07071
:20025400030202A7800B78FE122895E604F61480C6120046740A75F000C0E0C0F07401755D
:20027400F000C0E0C0F078FA122895E618181818860108860275F0001228B789828A83E43A
:20029400931228C7C0E0C0F01207E87FFA1228A102025A78FA122895E60886F01581221244
:2002B4000046740A75F000C0E0C0F0740175F000C0E0C0F078F7122895E61228C7C0E0C002
:2002D400F01207E87FFA1228A1227F081228A178F3122895E60886F07B007C001229A84584
:2002F400F0700302030D740075F00079F712289A1228B7742DF702031D740075F00079F764
:2003140012289A1228B7742BF778F3122895E60886F078FD122895F608A6F078F3122895BE
:20033400E60886F07B007C001229A845F0700302036B78FD122895E60886F01229A178F364
:20035400122895F608A6F018E60886F012298E18F608A6F0122997740175F00079F71228DF
:200374009A1228B778F3122895E60886F07BE87C031229142430C5F03400C5F0F718E60820
:2003940086F07BE87C0312290D78FD122895F608A6F0740275F00079F712289A1228B77849
:2003B400FD122895E60886F07B647C001229142430C5F03400C5F0F778F3122895E60886B8
:2003D400F07B647C0012290D78FD122895F608A6F0740375F00079F712289A1228B778FD18
:2003F400122895E60886F07B0A7C001229142430C5F03400C5F0F7740475F00079F71228F6
:200414009A1228B778FD122895E60886F07B0A7C0012290D2430C5F03400C5F0F77400757A
:20043400F00079F712289A1228B7E71228C7C0E0C0F01202B315811581740175F00079F70E
:2004540012289A1228B7E71228C7C0E0C0F01202B315811581740275F00079F712289A1267
:2004740028B7E71228C7C0E0C0F01202B315811581740375F00079F712289A1228B7E71254
:2004940028C7C0E0C0F01202B315811581740475F00079F712289A1228B7E71228C7C0E07C
:2004B400C0F01202B3158115817FF80228B0758E037481F5A8E5884401F5887400F53A7456
:2004D40000F56C740C75F000C0E0C0F0740075F000C0E0C0F0E53A1228C7C0E0C0F01207C0
:2004F400E87FFA1228A17400F511747075F017F55D85F05E746475F000F55385F054796383
:200514007A00E98AF0C0E0C0F0746475F000C0E0C0F012269A15811581158115811219E7D1
:200534001200C774C875F02DC0E0C0F012022115811581740075F000C0E0C0F0740175F04C
:2005540000C0E0C0F012014A158115811581158174D175F02DC0E0C0F012022115811581FA
:2005740074E875F003C0E0C0F01226CD1581158174BFF537E5114402F5111215EC74807505
:20059400F025C0E0C0F01226EA1581158179307A2AE98AF0C0E0C0F012270D158115811210
:2005B400112712121A121189121106120FDF1209B2120F0A120C7B120CF3120D301212ECDB
:2005D4001215171216C2121AFE1218C5121B95121BBE121C7C121EE11222B81209891215A7
:1705F400501215BA1215EC12077B120FB61223AB12241F0205B6222D
:07000300C0D0C0E002060BB3
:20060B00C0F0C083C082C000C001C002C003C004C005C006C00712063FD007D006D005D0D5
:20062B0004D003D002D001D000D082D083D0F0D0E0D0D032740875F000C0E0C0F074027562
:20064B00F000C0E0C0F01207BF1581158115811581F53D85F03E740875F000C0E0C0F07495
:20066B000175F000C0E0C0F01207BF1581158115811581F53F85F040E53F8540F05410C59E
:20068B00F05400C5F0F53BE53F8540F05420C5F05400C5F0F53CE53F8540F0540FC5F054A5
:2006AB0000C5F0F53F85F040E53F8540F07B087C0012296FF53F85F040E53D853EF0453FCD
:2006CB00C5F04540C5F0F53D85F03EE53B60030206EEE53D853EF07BFF7CFF1228F9F53D93
:2006EB0085F03EE53C70030206FF740F75F027F53D85F03EE53A1228C7C333C5F033C5F0FA
:20070B0079437A001228B7E53D853EF0F709A7F0E53A04F53A14E53A5403F53A740C75F04B
:20072B0000C0E0C0F0740075F000C0E0C0F0E53A1228C7C0E0C0F01207E87FFA1228A174FC
:20074B000175F000C0E0C0F01226CD15811581E53A1228C77B001228BE1229C845F0700369
:20076B0002077AE59054BFF590E5114480F51122E51675F0007B627C001229C845F0700398
:20078B000207A379437A2DE98AF0C0E0C0F012270D158115811211272278FB122895E6F591
:2007AB0013E513A2E09290A2E19291A2E29292A2E392932278F9122895E61228C7C0E0C0DE
:2007CB00F01207A41581158178FB122895E60886F0C0E0C0F0122749158115812278F712EE
:2007EB002895E61228C7C0E0C0F01207A41581158178F9122895E60886F0C0E0C0F008E62F
:20080B001228C7C0E0C0F012276A15811581158115812212278A74D075F000C0E0C0F01291
:20082B00279F15811581740775F000C0E0C0F012279F15811581749075F000C0E0C0F012BC
:20084B00279F158115811227972212278A74D075F000C0E0C0F012279F1581158174007500
:20086B00F000C0E0C0F012279F1581158112279712278A74D175F000C0E0C0F012279F15AF
:20088B008115817400F5717400F515E51575F0007B067C001229DB45F070030208CE800864
:2008AB00E51504F5151480E3E515794B7A0075F0001228B7C001C0021227C9D007D000F6FE
:2008CB000208AB7401F571E515794B7A0075F0001228B7C001C0021227C9D007D000F612BB
:2008EB0027972212278A74D075F000C0E0C0F012279F15811581740075F000C0E0C0F01212
:20090B00279F15811581740075F000C0E0C0F012279F15811581743075F000C0E0C0F01242
:20092B00279F15811581741275F000C0E0C0F012279F15811581740375F000C0E0C0F0123D
:20094B00279F15811581742575F000C0E0C0F012279F15811581740775F000C0E0C0F01206
:20096B00279F15811581740075F000C0E0C0F012279F158115811227972212085522E516CF
:20098B0075F0007B757C001229C845F070030209B179607A2CE98AF0C0E0C0F012270D1587
:2009AB0081158112112722E51675F0007B747C001229C845F07003020A5D74D975F02DC02B
:2009CB00E0C0F012270D15811581120B14F50D743A75F000C0E0C0F01227211581158112DC
:2009EB000B14F50C743A75F000C0E0C0F012272115811581120B14F50A12278A74D075F047
:200A0B0000C0E0C0F012279F15811581740075F000C0E0C0F012279F15811581E50A75F0F6
:200A2B0000C0E0C0F012279F15811581E50C75F000C0E0C0F012279F15811581E50D75F056
:200A4B0000C0E0C0F012279F15811581122797121127227F091228A1740075F00078FD1238
:200A6B002895F608A6F0122739C0E0C0F01227211581158178FC122895F67B0D7C0012295A
:200A8B00D145F07003020AC6801678FD122895E60886F012298E18F608A6F012299780C635
:200AAB0078FD122895E60886F079F612289A1228B778FC122895E6F7020A9578FD1228954A
:200ACB00E60886F079F612289A1228B77400F778FD122895E60886F07B007C001229C84521
:200AEB00F07003020AF974FF75F0FF020B0F79F612289AE98AF0C0E0C0F01227FD158115B9
:200B0B0081020B0F7FF70228B005810581058105810581740075F00078FD122895F608A67E
:200B2B00F078FD122895E60886F07B027C001229A845F07003020B86801678FD122895E63B
:200B4B000886F012298E18F608A6F012299780D178FD122895E60886F079FA12289A12284B
:200B6B00B7C001C002122739C0E0C0F012272115811581D007D000F6020B4578FD122895B5
:200B8B00E60886F079FA12289A1228B77400F7740075F00079FA12289A1228B7E7C39430C4
:200BAB001228C77B041228BE12296FC0E0C0F0740175F00079F812289A1228B7E7C394303A
:200BCB00D004D0034BC5F04CC5F01228C77FFB0228B005810581058105810581740075F096
:200BEB000078FD122895F608A6F078FD122895E60886F07B027C001229A845F07003020CD8
:200C0B004F801678FD122895E60886F012298E18F608A6F012299780D178FD122895E60872
:200C2B0086F079FA12289A1228B7C001C002122739C0E0C0F012272115811581D007D00089
:200C4B00F6020C0E78FD122895E60886F079FA12289A1228B77400F779FA12289AE98AF082
:200C6B00C0E0C0F01227FD158115817FFB0228B0E51675F0007B697C001229C845F07003F8
:200C8B00020CF274F875F02DC0E0C0F012270D15811581740075F000C0E0C0F01207A4158E
:200CAB00811581740475F000C0E0C0F0120A5E7B647C001228F9C0E0C0F012277815811531
:200CCB008115811581740475F000C0E0C0F012275815811581F55D85F05EE55D855EF0F543
:200CEB005B85F05C12112722E51154087003020D2FE55B855CF0122997F55B85F05C12290F
:200D0B008EE55B855CF07B007C001229E245F07003020D2FE55D855EF0F55B85F05CE51103
:200D2B004404F511220581E51714F51704E51775F0007B007C001229E245F07003020F075D
:200D4B007464F517120855740275F000794B7A001228B7E775F0007B047C0012297D78FEB6
:200D6B00122895F6E675F0007B0A7C001228F9F6740275F000794B7A001228B7C001C002A1
:200D8B00740275F000794B7A001228B7E7540F78FC12289526D007D000F6740175F000799B
:200DAB004B7A001228B7E775F0007B047C0012297D78FE122895F6E675F0007B0A7C0012DA
:200DCB0028F9F6740175F000794B7A001228B7C001C002740175F000794B7A001228B7E775
:200DEB00540F78FC12289526D007D000F6740075F000C0E0C0F01207A41581158174027582
:200E0B00F000794B7A001228B7C001C002740075F000C0E0C0F012274915811581D007D0A7
:200E2B000086037C001229C845F0602B740175F000794B7A001228B7C001C002740175F079
:200E4B0000C0E0C0F012274915811581D007D00086037C001229C845F07003020E96E51196
:200E6B004408F511742C75F001F55385F054743D75F000C0E0C0F0E51175F000C0E0C0F0ED
:200E8B0012276A1581158115811581740275F000794B7A001228B7C001C002740275F000E4
:200EAB00C0E0C0F012274915811581D007D00086037C001229C845F0602B740175F0007967
:200ECB004B7A001228B7C001C002740375F000C0E0C0F012274915811581D007D0008603C4
:200EEB007C001229C845F07003020F07E51154F7F511746475F000F55385F054158122E576
:200F0B001675F0007B647C001229C845F07003020FB5741075F02EC0E0C0F012270D15813C
:200F2B001581120B14F50E742D75F000C0E0C0F012272115811581120B14F50F742D75F0C5
:200F4B0000C0E0C0F012272115811581120B14F51012278A74D075F000C0E0C0F012279FE6
:200F6B0015811581740475F000C0E0C0F012279F15811581E50E75F000C0E0C0F012279F89
:200F8B0015811581E50F75F000C0E0C0F012279F15811581E51075F000C0E0C0F012279FEB
:200FAB001581158112279712112722E51675F0007B0D7C001229C845F07003020FDE793017
:200FCB007A2AE98AF0C0E0C0F012270D1581158112112722E51675F0007B2F7C001229C848
:200FEB0045F07003021105120855742F75F02EC0E0C0F0740475F000794B7A001228B7E73E
:20100B0075F000C0E0C0F0740575F000794B7A001228B7E775F000C0E0C0F0740675F00088
:20102B00794B7A001228B7E775F000C0E0C0F0740475F0001224567FF81228A1744075F006
:20104B002EC0E0C0F0740275F000794B7A001228B7E775F000C0E0C0F0740175F000794BC3
:20106B007A001228B7E775F000C0E0C0F0740075F000794B7A001228B7E775F000C0E0C0AA
:20108B00F0740475F0001224567FF81228A11211F5745075F02EC0E0C0F0740075F0007989
:2010AB00437A001228B7E70987F0C0E0C0F0740275F00079437A001228B7E70987F0C0E0B7
:2010CB00C0F0740475F00079437A001228B7E70987F0C0E0C0F0740675F00079437A001273
:2010EB0028B7E70987F0C0E0C0F0740575F0001224567FF61228A112112722E598540170E7
:20110B0003021122122739C0E0C0F012272115811581F51602112674FFF51622794B7A2AF8
:20112B00E98AF0C0E0C0F012270D158115812205810581740075F00078FD122895F608A690
:20114B00F078FD122895E60886F078F912289586030886041229A845F070030211848016D9
:20116B0078FD122895E60886F012298E18F608A6F012299780CB02116B158115812212113B
:20118B00901211CA22E559855AF012298EF55985F05A122997E559855AF0AB53AC5412299A
:2011AB00EB45F070030211C9740075F000F55985F05AE5114440F511C2977405F51422E55D
:2011CB0011544070030211F4E51414F51404E51475F0007B007C001229C845F070030211B8
:2011EB00F4D297E51154BFF51122E5904440F590E511548075F0007B007C001229C845F07A
:20120B0070030212130211FBE511547FF51122308DFDC28D438CDC2205810581740175F06E
:20122B000079637A001228B7E775F00078FD122895F608A6F018E60886F07B087C00122982
:20124B006F18F608A6F0740075F00079637A001228B778FD122895E60886F047158115812D
:20126B002274012563F563E43564F564E43565F5652212126C740275F00079637A00122821
:20128B00B7E775F000C0E0C0F01207A4158115811212232212126C12126C740275F000792A
:2012AB00637A001228B7E775F000C0E0C0F01207A4158115811212232278FB122895E675CA
:2012CB00F0007B047C0012297DF62430C5F03400C5F02278FB122895E6540F24301228C776
:2012EB0022E511540470030214D51211F512085512129FC0E0C0F0E5578558F0C0E0C0F022
:20130B00122778158115811581158112127DC0E0C0F0740475F000794B7A001228B7E77560
:20132B00F000C0E0C0F012276A158115811581158112127DC0E0C0F0740575F000794B7A5A
:20134B00001228B7E775F000C0E0C0F012276A158115811581158112127DC0E0C0F074068F
:20136B0075F000794B7A001228B7E775F000C0E0C0F012276A158115811581158112127D96
:20138B00C0E0C0F0740275F000794B7A001228B7E775F000C0E0C0F012276A158115811568
:2013AB0081158112127DC0E0C0F0740175F000794B7A001228B7E775F000C0E0C0F012273C
:2013CB006A158115811581158112127DC0E0C0F0740075F000794B7A001228B7E775F000FB
:2013EB00C0E0C0F012276A158115811581158112129FC0E0C0F0740075F00079437A001263
:20140B0028B7E70987F0C0E0C0F0122778158115811581158112129FC0E0C0F0740275F034
:20142B000079437A001228B7E70987F0C0E0C0F0122778158115811581158112129FC0E057
:20144B00C0F0740475F00079437A001228B7E70987F0C0E0C0F0122778158115811581158E
:20146B008112129FC0E0C0F0740675F00079437A001228B7E70987F0C0E0C0F0122778154A
:20148B0081158115811581E51154FBF511E5578558F012298EF55785F0581214D6740075E3
:2014AB00F000C0E0C0F01207A415811581740675F000C0E0C0F0E5578558F0C0E0C0F0125E
:2014CB002778158115811581158122E5578558F07B887C131229EB45F07003021516E5115C
:2014EB0054F7F511746475F000F55385F054743C75F000C0E0C0F074FF75F0FFC0E0C0F0B6
:20150B0012276A158115811581158122E51675F0007B727C001229C845F0700302154F7455
:20152B005D75F02EC0E0C0F0E5578558F0C0E0C0F0740275F00012245615811581158115C9
:20154B008112112722740E75F000C0E0C0F0740075F000C0E0C0F01207BF15811581158199
:20156B0015817BFF7C001229D145F0600EE511540175F0007B007C001229C845F0700302D1
:20158B0015B5E5114401F511740E75F000C0E0C0F0740075F000C0E0C0F01207BF15811552
:2015AB008115811581F5370215B974FFF53722740E75F000C0E0C0F0740075F000C0E0C046
:2015CB00F01207BF15811581158115817BFF7C001229C845F070030215EBE51154FEF511EF
:2015EB0022E53775F0007BFF7C001229D145F070030216C1E53775F0009016AD0228D0E507
:20160B006C04F56C140216C1E5116402F511E51154EFF5111200A0740075F000C0E0C0F085
:20162B00740175F000C0E0C0F012014A1581158115811581747375F02EC0E0C0F0120221C1
:20164B0015811581E5115402700302166B742A75F000C0E0C0F01202B3158115810216A40F
:20166B001200A012231F740075F000C0E0C0F0740075F000C0E0C0F012014A158115811569
:20168B00811581747B75F02EC0E0C0F012022115811581E5114410F5110216C10216C102F1
:2016AB0016C1AA16EF00A716DF001316BF000A167F000000C11622E51675F0007B737C00B3
:2016CB001229C845F07003021868740075F000C0E0C0F01207A415811581748475F02EC075
:2016EB00E0C0F0740075F000C0E0C0F012274915811581C0E0C0F0740175F000C0E0C0F0FE
:20170B0012274915811581C0E0C0F0740375F0001224567FFA1228A1740075F000C0E0C0CB
:20172B00F0120BDD1228C7C0E0C0F012276A1581158115811581743A75F000C0E0C0F012F3
:20174B00272115811581740175F000C0E0C0F0120BDD1228C7C0E0C0F012276A15811581C6
:20176B0015811581749775F02EC0E0C0F0740275F000C0E0C0F012274915811581C0E0C00B
:20178B00F0740375F000C0E0C0F012274915811581C0E0C0F0740375F0001224567FFA1231
:2017AB0028A1740275F000C0E0C0F0120BDD1228C7C0E0C0F012276A1581158115811581E4
:2017CB00743A75F000C0E0C0F012272115811581740375F000C0E0C0F0120BDD1228C7C02E
:2017EB00E0C0F012276A158115811581158174AA75F02EC0E0C0F0740075F000C0E0C0F029
:20180B0012274915811581C0E0C0F0740175F000C0E0C0F012274915811581C0E0C0F07423
:20182B000275F000C0E0C0F012274915811581C0E0C0F0740375F000C0E0C0F01227491525
:20184B00811581C0E0C0F0740575F0001224567FF61228A112186912231F12112722740095
:20186B0075F000C0E0C0F0122749158115817B637C001229C845F070030218A7743C75F01F
:20188B0000C0E0C0F0740175F000C0E0C0F012276A15811581158115810218C4743C75F0D5
:2018AB0000C0E0C0F074FF75F0FFC0E0C0F012276A158115811581158122E51675F0007BAE
:2018CB003D7C001229C845F070030219E6740075F000C0E0C0F01207A41581158174C075DD
:2018EB00F02EC0E0C0F0740075F000C0E0C0F012274915811581C0E0C0F0740175F000C0AE
:20190B00E0C0F012274915811581C0E0C0F0740375F0001224567FFA1228A174D275F02E99
:20192B00C0E0C0F0740275F000C0E0C0F012274915811581C0E0C0F0740375F000C0E0C0E7
:20194B00F012274915811581C0E0C0F0740375F0001224567FFA1228A174E475F02EC0E047
:20196B00C0F0740475F000C0E0C0F0122758158115817B647C00122914C0E0C0F0740275DD
:20198B00F0001224561581158115811581743C75F000C0E0C0F0122749158115817B017C5D
:2019AB00001229C845F070030219CE740275F02FC0E0C0F0740175F000122456158115819C
:2019CB000219E3740B75F02FC0E0C0F0740175F0001224561581158112112722740075F0C4
:2019EB0000C0E0C0F01207A415811581743D75F000C0E0C0F012274915811581F511740411
:201A0B0075F000C0E0C0F012275815811581F55D85F05EE55D855EF0F55B85F05C740675FF
:201A2B00F000C0E0C0F012275815811581F55785F05879697A00E98AF0C0E0C0F0742E755F
:201A4B00F000C0E0C0F012269A158115811581158179667A00E98AF0C0E0C0F0E5578558EC
:201A6B00F0C0E0C0F012269A158115811581158179667A00E98AF0C0E0C0F079697A00E9A0
:201A8B008AF0C0E0C0F01225EC158115811581158179667A00E98AF0C0E0C0F0746475F0AD
:201AAB0000C0E0C0F012269A1581158115811581796D7A00E98AF0C0E0C0F079667A00E94C
:201ACB008AF0C0E0C0F01225AB158115811581158179637A00E98AF0C0E0C0F0796D7A008E
:201AEB00E98AF0C0E0C0F012265D158115811581158122E51675F0007B6E7C001229C8450C
:201B0B00F07003021B94741275F02FC0E0C0F012270D158115811227397B797C001229C8E5
:201B2B0045F07003021B91E51154F7F511740075F000F55785F058740075F000C0E0C0F0E2
:201B4B001207A415811581740675F000C0E0C0F0740075F000C0E0C0F0122778158115815C
:201B6B001581158179637A00E98AF0C0E0C0F0746475F000C0E0C0F012269A158115811585
:201B8B0081158112214E12112722E51675F0007B3F7C001229C845F07003021BBD794F7AD9
:201BAB002AE98AF0C0E0C0F012270D1581158112112722E51675F0007B637C001229C8455D
:201BCB00F07003021C7B120855742575F02FC0E0C0F0740475F000794B7A001228B7E775AA
:201BEB00F000C0E0C0F0740575F000794B7A001228B7E775F000C0E0C0F0740675F0007999
:201C0B004B7A001228B7E775F000C0E0C0F0740475F0001224567FF81228A1743675F02F6E
:201C2B00C0E0C0F0740275F000794B7A001228B7E775F000C0E0C0F0740175F000794B7A8B
:201C4B00001228B7E775F000C0E0C0F0740075F000794B7A001228B7E775F000C0E0C0F048
:201C6B00740475F0001224567FF81228A112112722E51675F0007B617C001229C845F070D2
:201C8B0003021EE012222279667A00E98AF0C0E0C0F0740175F000C0E0C0F012269A158142
:201CAB0015811581158179637A00E98AF0C0E0C0F079667A00E98AF0C0E0C0F01225BE1538
:201CCB008115811581158179667A00E98AF0C0E0C0F079637A00E98AF0C0E0C0F012265D0C
:201CEB00158115811581158179637A00E98AF0C0E0C0F0746475F000C0E0C0F012269A1504
:201D0B0081158115811581740075F000F56185F062E5618562F0AB57AC581229DB45F07091
:201D2B0003021EDD8012E5618562F012298EF56185F06212299780D9740D75F000C0E0C082
:201D4B00F012213C15811581740A75F000C0E0C0F012213C1581158112129FC0E0C0F012FA
:201D6B00275815811581744675F02FC0E0C0F0E5618562F0C0E0C0F0740275F0001224563B
:201D8B001581158115811581744A75F02FC0E0C0F012127DC0E0C0F012274915811581C0DF
:201DAB00E0C0F012127DC0E0C0F012274915811581C0E0C0F012127DC0E0C0F01227491511
:201DCB00811581C0E0C0F0740475F0001224567FF81228A1745A75F02FC0E0C0F012127D83
:201DEB00C0E0C0F012274915811581C0E0C0F012127DC0E0C0F012274915811581C0E0C08B
:201E0B00F012127DC0E0C0F012274915811581C0E0C0F0740475F0001224567FF81228A11D
:201E2B00746A75F02FC0E0C0F012129FC0E0C0F012275815811581C0E0C0F0740275F000DA
:201E4B001224561581158115811581746E75F02FC0E0C0F012129FC0E0C0F0122758158193
:201E6B001581C0E0C0F0740275F0001224561581158115811581747275F02FC0E0C0F012D6
:201E8B00129FC0E0C0F012275815811581C0E0C0F0740275F00012245615811581158115EB
:201EAB0081747675F02FC0E0C0F012129FC0E0C0F012275815811581C0E0C0F0740275F0CD
:201ECB00001224561581158115811581122102021D3112112722E51675F0007B787C001241
:201EEB0029C845F0700302210112222279667A00E98AF0C0E0C0F0740175F000C0E0C0F08E
:201F0B0012269A158115811581158179637A00E98AF0C0E0C0F079667A00E98AF0C0E0C067
:201F2B00F01225BE158115811581158179667A00E98AF0C0E0C0F079637A00E98AF0C0E0F4
:201F4B00C0F012265D158115811581158179637A00E98AF0C0E0C0F0746475F000C0E0C033
:201F6B00F012269A1581158115811581740075F000F56185F062E5618562F0AB57AC581201
:201F8B0029DB45F070030220FE8012E5618562F012298EF56185F06212299780D9740D75A4
:201FAB00F000C0E0C0F012213C15811581740A75F000C0E0C0F012213C1581158112129FAA
:201FCB00C0E0C0F012275815811581747A75F02FC0E0C0F0E5618562F0C0E0C0F0740275BF
:201FEB00F000122456158115811581158112127DC0E0C0F01227491581158112127DC0E022
:20200B00C0F01227491581158112127DC0E0C0F01227491581158112127DC0E0C0F012278E
:20202B00491581158112127DC0E0C0F01227491581158112127DC0E0C0F012274915811563
:20204B0081747E75F02FC0E0C0F012129FC0E0C0F012275815811581C0E0C0F0740275F023
:20206B00001224561581158115811581748275F02FC0E0C0F012129FC0E0C0F012275815DE
:20208B00811581C0E0C0F0740275F0001224561581158115811581748675F02FC0E0C0F031
:2020AB0012129FC0E0C0F012275815811581C0E0C0F0740275F000122456158115811581CC
:2020CB001581748A75F02FC0E0C0F012129FC0E0C0F012275815811581C0E0C0F074027572
:2020EB00F0001224561581158115811581122102021F961211272205811228417B137C009E
:20210B001229C845F0700302213978FE122895E61228C77B111228BE1229D145F070030247
:20212B00213912284178FE122895F602211515812278FB122895E6F5133099FDC299E5134B
:20214B00F59922748E75F02FC0E0C0F012270D1581158179187A00E98AF0C0E0C0F0741E1C
:20216B0075F000C0E0C0F01228531581158115811581740075F000C0E0C0F01207A415813E
:20218B001581740075F000F56185F062E5618562F079187A001228B7E775F0007B007C003C
:2021AB001229D145F070030221FC8012E5618562F012298EF56185F06212299780CEE56136
:2021CB008562F02408C5F03400C5F0C0E0C0F0E5618562F079187A001228B7E775F000C0DE
:2021EB00E0C0F012276A15811581158115810221B7E5618562F02408C5F03400C5F0C0E0E8
:20220B00C0F0740075F000C0E0C0F012276A1581158115811581220581740D75F000C0E0B1
:20222B00C0F012213C15811581740A75F000C0E0C0F012213C15811581740075F000C0E001
:20224B00C0F01207A415811581740075F000F56185F062E5618562F02408C5F03400C5F0ED
:20226B00C0E0C0F01227491581158178FE122895F67B007C001229D145F070030222B58016
:20228B0012E5618562F012298EF56185F06212299780C078FE122895E61228C7C0E0C0F080
:2022AB001227211581158102228C158122740075F000C0E0C0F01207A415811581743C75EE
:2022CB00F000C0E0C0F0122749158115817B017C001229C845F0700302231EE5B0540875B9
:2022EB00F0007B007C001229C845F0700302230EE5114408F511742C75F001F55385F054AF
:20230B0002231EE51154F7F511746475F000F55385F05422740075F000C0E0C0F01207A4D2
:20232B0015811581743C75F000C0E0C0F0122749158115817B017C001229C845F0700302AE
:20234B00237D740775F000C0E0C0F0740175F000C0E0C0F012014A1581158115811581744F
:20236B004D75F000C0E0C0F01202B3158115810223AA740775F000C0E0C0F0740175F00084
:20238B00C0E0C0F012014A1581158115811581744175F000C0E0C0F01202B31581158122AE
:2023AB00E5115402700302241E1211F5740075F000C0E0C0F0740075F000C0E0C0F0120192
:2023CB004A1581158115811581E56C5403F56CE56C243175F000C0E0C0F01202B31581157A
:2023EB0081742075F000C0E0C0F01202B315811581E56C75F000C333C5F033C5F079437A96
:20240B00001228B7E70987F0C0E0C0F01202DE1581158122E5115410700302245574007598
:20242B00F000C0E0C0F0740175F000C0E0C0F012014A1581158115811581E5578558F0C0A9
:20244B00E0C0F01202DE158115812223F42581F8868208868308E4FEFF93700122B4255596
:20246B00A3E493B42D06430780A3E493B4300343074024D0B40A00500CCE75F00AA42EFEE0
:20248B00A3E49380EDE493B46413E60886F030F70843072012299EA6F018F68003B47505DD
:2024AB0043070A801CB478054307108014B46F0B430708800C122727A3809BB46262430716
:2024CB00027A00C004C005C006C007AB0753031F7C00E60886F012293CA6F018F6EDD00779
:2024EB00D006D005D0042430B43A0040022407C0E00AE645F070CCA902EF30E506742D123A
:20250B0027270A12258CD0E0122727D9F90808EF30E7A5EAC39E50A074201227270A80F34C
:20252B00B4630BAA0112258CE612272780DFB4732BC082C08386820886837A00E493600416
:20254B00A30A80F8868318868212258CE493A3600512272780F6D083D08280B1B469198678
:20256B00017A00E76004090A80F912258C8601E7609B1227270980F7F97A0112258CE98052
:20258B00A8EE601B8FF020F716C002EAC39E500D742030F60274301227270A80EED00222DD
:2025AB001226B77A04C3E637F60809DAF9E4F5F092E0221226B77A04C3E697F60809DAF905
:2025CB0080EB1226AFC37A04E633F608DAFA80DD1226AF7A04C82AC8C318E613F6DAFA80D8
:2025EB00CC1226B7AB00A8817F041228A108AC001226601226C3A8031225DE5007786DA9F7
:20260B00041225AEA80312266C600CA8041225D0A80412266C70DFA803796D1226607FFC15
:20262B000228B01226B7AB00AC011226C37D21C3A8031225D1DD028033786D1225D1786DFB
:20264B00A90412267B20E7E7786DA9041225C1D380DE1226B77A04E7F60908DAFA221226DD
:20266B00AF7A0475F000E6700308DAFA221226B77A04E82AF8E92AF9181987F0E6B5F006AA
:20268B00DAF6E4F5F02274FF40F904F5F00422E58124FBF987001226C587000909E7F60839
:2026AB0009E7F622E58124FBF8860022E58124FBF886011818860022786D7A04760008DA4B
:2026CB00FB2278FB1228958603088604BB0004BC00012279E5A3D9FD1BBBFFF01C80F47833
:2026EB00FB1228958603088604748075F07012293C12299E758921F58DF58B75885975984D
:20270B00522278FB1228958682088683E493602D122727A380F678FB122895E63099FDC2B2
:20272B0099F599B40A17740D80F2E430980C3098FDC298E599B40D02740A75F0002278FB0F
:20274B001228958682088683E075F0002278FB1228958682088683E0F5F0A3E0C5F022782D
:20276B00F9122895868208868308E6F02278F9122895868208868308E608F0A3E6F022D2C1
:20278B00951227EFC2951227F5C29422C2951227EFD2952278FB122895E67F0830E704D2D0
:2027AB00958002C2951227EF23C294DFEFD2951227EF3095001227F5C2941227F5227F0882
:2027CB007400D2951227EFA29533C294DFF6C0E0D295E571B40002C2951227EFC294D0E0BE
:2027EB0075F00022D2943094FD22000022000000002278FB1228958601E4FBFCFFE709B473
:20280B002D030FE709C39430B40A005012FA740A75F0001228F92AFBE5F03400FC80E4EB4E
:20282B008CF0DF0302299E2278FB122895E63099FDC299F5992274FFF5F030980A3098FD5C
:20284B00C298E59975F0002278FB122895860418188601E4FD122739B408028003B47F16AE
:20286B00ED60F21D7408122727742012272774081227271980DF122727F724F36006090DE3
:20288B00EDB504D1E4F7F5F0ED22C82581C822C92581C97A0022D083D082CF2581F581CF5C
:2028AB00C082C08322CF2581F581CF2229F9E5F03AFA227C00CB30E7011CCB2275F0003040
:2028CB00E70215F022FDE493A3FEE493A3FF4E7009E493FE740193FF800BE493A3B5050B02
:2028EB00E493B5F0068F838E82E473A380D8FEEBA4FD8EF0ECA4FCEB8EF0A4C5F02C2DC5C3
:20290B00F02212293C8EF0ED22C0F0C0E0E5F06C5480FF8CF030F707EB12299EACF0FBD05D
:20292B00E0D0F030F70312299EBF800512293C8062C002C001AAF0F97E007D007F11C3E9FF
:20294B0033F9EA33FADF08F5F0E9D001D00222ED33FDEE33FEC3ED9BF5F0EE9C40E0ADF0FC
:20296B00FED380DBBB000122C333C5F033C5F0DBF722BB000122C3C5F013C5F013DBF72296
:20298B0012298E04700205F02212299714B4FF0215F022122997F4C5F0F4C5F0221229FB98
:2029AB004029801E1229FB40227017801E1229FB40107017800C1229FB50108005122A0F49
:2029CB006009E4F5F022122A0F60F7E4F5F00422122A0F40F680EB122A0F40EF70E480EBE2
:2029EB00122A0F40DD70E480D9122A0F50DD80D2C39BC5F09C20E70720D207C345F02220FD
:202A0B00D2F9D322C5F0C39C7003E5F09B22FBE493CB22FCE493FB740193CC22FAE493F9A5
:202A2B00740193CA220A0A4D696E694C4F474745522056332E3020283F2068656C702900B6
:202A4B000A3E3E000A0A48454C50204D454E55202020202020202020202020202020200A49
:202A6B002F207072696E7420616E616C6F672072656164696E672020202020202020202003
:202A8B002020202020200A742054494D452073657420202020202020202020202020202052
:202AAB00200A64204441544520736574202020202020202020202020202020200A63204303
:202ACB006C6F636B20646973706C6179202020202020202020202020202020200A7320731C
:202AEB0065742053544152542F53544F50207265636F7264696E672074696D6520202020A3
:202B0B002020202020202020202020200A692073616D706C696E6720496E74657276616CD7
:202B2B00202020202020202020202020202020200A3D20646973706C6179207365747469E4
:202B4B006E6720706172616D6574657273202020202020202020202020202020200A7220A5
:202B6B006E756D626572206F66207265636F7264202020202020202020202020202020202D
:202B8B000A62207465726D696E616C20636F6E6E656374696F6E20202020202020202020B2
:202BAB002020202020200A6E204E6577207265636F72642020202020202020202020202049
:202BCB002020200A6120414C4C20726561643A2073616D706C65207265616C2D74696D65EE
:202BEB0020616E642064617461202020202020202020202020202020200A7820526561649F
:202C0B0020416C6C3A2073616D706C6520616E642064617461202020202020202020202027
:202C2B0020202020200A752041626F7574204D696E694C4F474745522056332E302020207B
:202C4B00202020202020202020202020200A3F2068656C70000A4D696E694C4F4747455260
:202C6B002077617320646573696E67656420627920576963686974205349524943484F5473
:202C8B0045203238204A756E65203230303320202020202020202020202020202020200A99
:202CAB004170706C696564205068797369637320446570742E204B4D49544C20202020202B
:202CCB002020202020202020202020200A6669726D7761726520757064617465643A20326F
:202CEB0035204A756E65203230303420202020202020202020202020202020200A55524CDF
:202D0B003A207777772E6B6D69746C2E61632E74682F7E6B7377696368697420656D6169CF
:202D2B006C3A206B73776963686974406B6D69746C2E61632E7468000A20312020202032F2
:202D4B002020202033202020203420202020352020202036202020203720202020382020E7
:202D6B002020392020203130202031312020313220202020202020202020202020202020C9
:202D8B00202020200A494E312B20494E312D20494E322B20494E322D20494E332B20494EA0
:202DAB00332D20494E342B20494E342D202D3556202B35562020305620202B56004D696E21
:202DCB00694C4F47470045522056332E30000A656E7465722063757272656E742074696D03
:202DEB00652048483A4D4D3A5353203E000A20696E74657276616C20312D36303020736506
:202E0B0063203E20000A656E7465722063757272656E7420646174652044442D4D4D2D59C8
:202E2B0052203E000A253032782D253032782D253032782000253032783A253032783A25BF
:202E4B003032782000202564202564202564202564000A2575207265636F7264732061761C
:202E6B0061696C61626C650078302E316D5620005265636F72643D20000A5354415254201F
:202E8B00253032643A25303264203E000A53544F502020253032643A25303264203E000AB1
:202EAB0020253032643A2530326420253032643A25303264000A2053544152542025303248
:202ECB00643A25303264000A2053544F502020253032643A25303264000A2053414D504CF7
:202EEB00494E4720494E54455256414C2873656329203D202575000A204D414E55414C00D9
:202F0B000A204155544F000A204E6577207265636F72643F28592F4E29000A253032782DB4
:202F2B00253032782D253032782000253032783A253032783A2530327820002025640020E1
:202F4B00253032782D253032782D253032780020253032783A253032783A2530327800205E
:202F6B002564002025640020256400202564002025640020256400202564002025640020FE
:202F8B002564000A3C2D2D20456E746572206465736372697074696F6E20746578742028EE
:172FAB006D61782033302063686172616374657273292D2D3E0A003B
:00000001FF
